:020000040000FA
:02000000AD2928
:080008000B1923289B000730AF
:100010006200030EA200061C122881019801030150
:1000200062001C28010881019A00180899000B1928
:10003000990A0F14403062008B100B11220E8300BE
:100040009B0E1B0E09000B11980F090009001030C0
:10005000A50012089600130897009201930108006A
:100060009109910A03199003900900342720940103
:1000700095010310970D960D950D940D100814021F
:10008000031D442811081502031C4D281108950270
:10009000031C9403100894020314930D920D031093
:1000A000970D960D950D940D10081402031D5A28F6
:1000B00011081502031C632811089502031C940300
:1000C000100894020314930D920D0310970D960DD2
:1000D000950D940D10081402031D702811081502C7
:1000E000031C792811089502031C9403100894023C
:1000F0000314930D920D0310970D960D950D940D0D
:1001000010081402031D862811081502031C8F28ED
:1001100011089502031C9403100894020314930D14
:10012000920D0310970D960D950D940D1008140265
:10013000031D9C2811081502031CA528110895020F
:10014000031C9403100894020314930D920D0310E2
:10015000970D960D950D940D10081402031DB228ED
:1001600011081502031CBB2811089502031C9403F7
:10017000100894020314930D920D0310970D960D21
:10018000950D940D10081402031DC82811081502BE
:10019000031CD12811089502031C94031008940233
:1001A0000314930D920D0310970D960D950D940D5C
:1001B00010081402031DDE2811081502031CE7288D
:1001C00011089502031C9403100894020314930D64
:1001D000920D0310970D960D950D940D10081402B5
:1001E000031DF42811081502031CFD2811089502AF
:1001F000031C9403100894020314930D920D031032
:10020000970D960D950D940D10081402031D0A29E3
:1002100011081502031C132911089502031C9403ED
:10022000100894020314930D920D0310970D960D70
:10023000950D940D10081402031D202911081502B4
:10024000031C292911089502031C94031008940229
:100250000314930D920D0310970D960D950D940DAB
:1002600010081402031D362911081502031C3F292A
:1002700011089502031C9403100894020314930DB3
:10028000920D0310970D960D950D940D1008140204
:10029000031D4C2911081502031C5529110895024C
:1002A000031C9403100894020314930D920D031081
:1002B000970D960D950D940D10081402031D6229DB
:1002C00011081502031C6B2911089502031C9403E5
:1002D000100894020314930D920D0310970D960DC0
:1002E000950D940D10081402031D782911081502AC
:1002F000031C812911089502031C94031008940221
:100300000314930D920D0310970D960D950D940DFA
:1003100010081402031D8E2911081502031C9729C9
:1003200011089502031C9403100894020314930D02
:10033000920D0800110893070318920A10089207FB
:1003400008002720960C970C03189A21920C930C06
:10035000940C950CA50BA229080081014030620085
:100360008C018F010C3065003F3066000617861344
:100370008510061ECA2A392390080319C62964006D
:100380000630EB22110811020319D3291030A10005
:1003900002309C0000309D0004309E0000309F0021
:1003A0000230A000DF292030840005308D00831347
:1003B0000D08EB221108800084038D0BD8291D083D
:1003C0001F0293001C08031C1C0A1E0292009001CD
:1003D0001F30910036201308A100B0308B0064005C
:1003E0008730A300A4010F100430650085150516A1
:1003F000810198010530180203180E2A051EFA29FA
:100400004E230F18EF290618EF29103093002730DC
:10041000920036201308A3001208A40019308D00A2
:1004200064000F1C102A0F108D0B102A0830650075
:100430000F114030620005158101980189016400A7
:10044000051A4E230F1C1F2A0F100F1D452A2308C3
:10045000930024089200A1219508051C392AB03C7C
:100460001408031C140A043C031C452A03018C01D4
:100470009C2A583C1408031C140A023C031C452AFD
:100480000514851003018C019C2A0510861C002B85
:10049000061D142B1A08FA3C1908031C190A003C03
:1004A0000318A32A1A08E23C1908031C190A043C81
:1004B000031CA32A1D081A0293001C08031C1C0A13
:1004C000190292000318672A92019301772A1A08E9
:1004D0001F021908031C190A1E020318772A1D0897
:1004E0001F0293001C08031C1C0A1E0292009001AC
:1004F0002108910036201F301302031C812A1F306F
:100500009300861E992A131A8B2A85108F1844236C
:100510008F1093098F2A85148F1C44238F14031086
:10052000130D1F398C001E3C1F3003198C000C0862
:100530009C2A13091F398C00861D282B20020318C2
:100540008C011F308C060F111F300C06031DB02AC2
:1005500086130617861E85140516810198011F2A29
:10056000861E851005168101980110308D002030FF
:100570008E00861706130F18242A0E080C02C030AE
:1005800003198606051A4E238E0BBD2A64008D0BB7
:10059000B72AB52A8B011030A10001308900023042
:1005A0009C00F222890A00309D00F222890A043060
:1005B0009E00F222890A00309F00F222890A01304F
:1005C000A000F2223923063089001108F2226400CB
:1005D000061EE72AAD29890083160814831208082D
:1005E0009100080088008316081555308900AA304C
:1005F000890088146400081EFA2A88018312080002
:100600008B13861306178510013089001908F22212
:10061000890A1A08F2223923063089001108F222C9
:100620006400861C102BAD298B13861306178510CA
:10063000033089001908F222890A1A08F2223923A4
:10064000063089001108F2226400061D242BAD2912
:100650008B13861306178510053089000C08F222CB
:100660003923063089001108F2226400861D352BDB
:10067000AD2905308D00910190010D08EB22900409
:1006800091078D0B3D2B0800FF308D0082308E00CE
:100690008D0B482B64008E0B482B080047306200FE
:0E06A000051201089100180890000F150800BF
:02400E00F63F7B
:00000001FF
